:020000040000FA
:04080000DBEF06F034
:1008100003B20AEF05F0F2B428EF05F09EB030EF16
:1008200005F09EB238EF05F0F2A81AEF04F0F2B22C
:100830001CEF04F08AEF06F0CD90F2929EA026EF16
:1008400004F00101533F26EF04F0542BAEC1B2F186
:10085000AFC1B3F1B0C1B4F1B1C1B5F1AAC1AEF14C
:10086000ABC1AFF1ACC1B0F1ADC1B1F1A6C1AAF15C
:10087000A7C1ABF1A8C1ACF1A9C1ADF1A2C1A6F16C
:10088000A3C1A7F1A4C1A8F1A5C1A9F19EC1A2F17C
:100890009FC1A3F1A0C1A4F1A1C1A5F19AC19EF18C
:1008A0009BC19FF19CC1A0F19DC1A1F196C19AF19C
:1008B00097C19BF198C19CF199C19DF1CECF96F162
:1008C000CFCF97F153C198F154C199F1CF6ACE6A55
:1008D0000101536B546B9E90CD800FBC0F8E0FBAED
:1008E00075EF04F00F8A8AEF06F00F8C0FBEB1EFA0
:1008F00004F096C19AF197C19BF198C19CF199C1FE
:100900009DF19AC19EF19BC19FF19CC1A0F19DC137
:10091000A1F19EC1A2F19FC1A3F1A0C1A4F1A1C107
:10092000A5F1A2C1A6F1A3C1A7F1A4C1A8F1A5C1D7
:10093000A9F1A6C1AAF1A7C1ABF1A8C1ACF1A9C1A7
:10094000ADF1AAC1AEF1ABC1AFF1ACC1B0F1ADC177
:10095000B1F1AEC1B2F1AFC1B3F1B0C1B4F1B1C147
:10096000B5F101015E6B5F6B606B616B96515E2749
:1009700097515F2398516023995161239A515E27C3
:100980009B515F239C5160239D5161239E515E27A3
:100990009F515F23A0516023A1516123A2515E2783
:1009A000A3515F23A4516023A5516123A6515E2763
:1009B000A7515F23A8516023A9516123AA515E2743
:1009C000AB515F23AC516023AD516123AE515E2723
:1009D000AF515F23B0516023B1516123B2515E2703
:1009E000B3515F23B4516023B5516123D890010105
:1009F000613360335F335E33D8900101613360331C
:100A00005F335E33D8900101613360335F335E330F
:100A10008AEF06F00392ABB2AB98AB88030103EE0A
:100A200000F080517F0BE92604C0EFFF802B81513D
:100A3000805D700BD8A48B8200008051815D700BAB
:100A4000D8A48B9281518019D8B407908AEF06F010
:100A5000F2940101453F8AEF06F0462B8AEF06F03B
:100A60009E900101533F8AEF06F0542B8AEF06F067
:100A70009E92C3CF55F1C4CF56F1C28207B4A3EF03
:100A800005F047C14BF148C14CF149C14DF14AC194
:100A90004EF15EC162F15FC163F160C164F161C199
:100AA00065F196C1B6F197C1B7F198C1B8F199C196
:100AB000B9F19AC1BAF19BC1BBF19CC1BCF19DC116
:100AC000BDF19EC1BEF19FC1BFF1A0C1C0F1A1C1E6
:100AD000C1F1A2C1C2F1A3C1C3F1A4C1C4F1A5C1B6
:100AE000C5F1A6C1C6F1A7C1C7F1A8C1C8F1A9C186
:100AF000C9F1AAC1CAF1ABC1CBF1ACC1CCF1ADC156
:100B0000CDF1AEC1CEF1AFC1CFF1B0C1D0F1B1C125
:100B1000D1F1B2C1D2F1B3C1D3F1B4C1D4F1B5C1F5
:100B2000D5F1010155515B2756515C23E86A5D23DD
:100B30000E2EA3EF05F05CC157F15DC158F15B6B60
:100B40005C6B5D6B078E0201002F8AEF06F03C0E96
:100B5000006F00C10CF101C10DF102C10EF103C122
:100B60000FF104C110F105C111F106C112F107C165
:100B700013F108C114F109C115F10AC116F10BC135
:100B800017F134C135F101018A67CEEF05F08B67AB
:100B9000CEEF05F08C67CEEF05F08D67D2EF05F054
:100BA00002EF06F08EC100F18FC101F190C102F198
:100BB00091C103F10101010E046F000E056F000EDB
:100BC000066F000E076F1DEC15F000C18EF101C11C
:100BD0008FF102C190F103C191F10067F7EF05F0C9
:100BE0000167F7EF05F00267F7EF05F0036702EF23
:100BF00006F08AC18EF18BC18FF18CC190F18DC14D
:100C000091F10F80D57ED5BE69D0D6CF47F1D7CF31
:100C100048F145C149F1E86AE8CF4AF1109047C16F
:100C200000F148C101F149C102F14AC103F10101DA
:100C30000A0E046F000E056F000E066F000E076FA0
:100C40001DEC15F003AF1080010154A734EF06F03E
:100C50000F9A0F9C0F9E0101000E5E6F600E5F6F7A
:100C60003D0E606F080E616F010147BF44EF06F053
:100C7000486744EF06F0496744EF06F04A6744EFDF
:100C800006F0F28869EF06F0F2985E6B5F6B606BBE
:100C9000616B966B976B986B996B9A6B9B6B9C6B6C
:100CA0009D6B9E6B9F6BA06BA16BA26BA36BA46BE8
:100CB000A56BA66BA76BA86BA96BAA6BAB6BAC6B98
:100CC000AD6BAE6BAF6BB06BB16BB26BB36BB46B48
:100CD000B56BD76AD66A0101456B466B0CC100F152
:100CE0000DC101F10EC102F10FC103F110C104F1F8
:100CF00011C105F112C106F113C107F114C108F1C8
:100D000015C109F116C10AF117C10BF135C134F152
:100D10008AEF06F002C0E0FF005001C0D8FF1000CB
:100D2000A6B290EF06F00CC0A9FF0BC0A8FFA69ECC
:100D3000A69CA684F29E550EA76EAA0EA76EA6824A
:100D4000F28EA694A6B2A2EF06F00C2A1200A96EAB
:100D5000A69EA69CA680A8500C2A120004012C0E68
:100D6000826F8FEC08F018EC16F00C50A7EC06F030
:100D7000E8CF00F10C50A7EC06F0E8CF01F101AF8D
:100D8000C7EF06F00101FF0E026FFF0E036FBBEC11
:100D900015F02967D3EF06F00401200E826F8FEC67
:100DA00008F0D8EF06F004012D0E826F8FEC08F0EA
:100DB000E5EC13F01200076A0F6A106A0F010E0EBD
:100DC000C16E860EC06E030EC26E0F01896A190EC7
:100DD000926E080E8A6EF10E936E8B6A800E946E80
:100DE000F18E0E6A01015B6B5C6B5D6B576B586B30
:100DF000F29A0101476B486B496B4A6B4B6B4C6B2A
:100E00004D6B4E6B4F6B506B516B526B456B466B22
:100E1000D76AD66A0F01280ED56EF28A9D90B00E61
:100E2000CD6E01015E6B5F6B606B616B626B636BC0
:100E3000646B656B666B676B686B696B536B546B4C
:100E4000CF6ACE6A0F9A0F9C0F9E9D80760ECA6E57
:100E50009D8202013C0E006FCC6A160EA7EC06F0D4
:100E6000E8CF00F1170EA7EC06F0E8CF01F1180E5D
:100E7000A7EC06F0E8CF02F1190EA7EC06F0E8CFD8
:100E800003F1010103AF5FEF07F018EC16F0160E47
:100E90000C6E00C10BF090EC06F0170E0C6E01C149
:100EA0000BF090EC06F0180E0C6E02C10BF090ECFB
:100EB00006F0190E0C6E03C10BF090EC06F000C1A9
:100EC0008AF101C18BF102C18CF103C18DF100C126
:100ED0008EF101C18FF102C190F103C191F11A0E9F
:100EE000A7EC06F0E8CF00F11B0EA7EC06F0E8CF68
:100EF00001F11C0EA7EC06F0E8CF02F11D0EA7ECE5
:100F000006F0E8CF03F1010103AFB5EF07F018ECED
:100F100016F01A0E0C6E00C10BF090EC06F01B0ED2
:100F20000C6E01C10BF090EC06F01C0E0C6E02C1B1
:100F30000BF090EC06F01D0E0C6E03C10BF090EC64
:100F400006F01A0EA7EC06F0E8CF00F11B0EA7EC96
:100F500006F0E8CF01F11C0EA7EC06F0E8CF02F195
:100F60001D0EA7EC06F0E8CF03F100C192F101C11C
:100F700093F102C194F103C195F1240EAC6E900E71
:100F8000AB6E240EAC6E080EB86E80B6E6EF07F0BE
:100F90001E0EA7EC06F0E8CF00F11F0EA7EC06F03E
:100FA000E8CF01F100C1E8FFFF0A10E001C1E8FF4E
:100FB000FF0A0CE01E0EA7EC06F0E8CFAFFF1F0EF5
:100FC000A7EC06F0E8CFB0FFEAEF07F0000EB06E36
:100FD0001F0EAF6E0401806B816B0F01900EAB6E24
:100FE0000F019D8A0301806B816BC26B8B9207900E
:100FF0000001F28EF28C07B095EF12F00FB076EF91
:101000000DF00301805181197F0BD8B495EF12F0D8
:1010100013EE00F081517F0BE126812BE7CFE8FF33
:10102000E00BD8B495EF12F023EE82F0C2513F0BE3
:10103000D926E7CFDFFFC22BDF50780AD8A495EF7F
:1010400012F007808EC100F18FC101F190C102F151
:1010500091C103F10101040E046F000E056F000E33
:10106000066F000E076F1DEC15F000AF41EF08F0A2
:101070000101030E8E6F000E8F6F000E906F000E39
:10108000916F03018251720AD8B476EF0DF082514C
:10109000520AD8B476EF0DF08251750AD8B476EFC3
:1010A0000DF08251630AD8B451EF0FF08251690AF2
:1010B000D8B434EF0AF082517A0AD8B447EF0BF073
:1010C0008251490AD8B4D3EF09F08251500AD8B4FA
:1010D000F1EF08F08251700AD8B434EF09F0825170
:1010E000540AD8B45FEF09F08251740AD8B4A5EF5E
:1010F00009F08251730AD8B4A6EF0CF08251530A5A
:10110000D8B40BEF0DF08251620AD8B4A3EF08F007
:101110008251420AD8B4DEEF08F086EF0FF00401E6
:1011200014EE00F080517F0BE12682C4E7FF802B94
:10113000120004010D0E826F8FEC08F00A0E826F10
:101140008FEC08F012008351610AD8A486EF0FF0EB
:101150008451750AD8A486EF0FF08551640AD8A48B
:1011600086EF0FF086C32AF187C32BF188C32CF1D9
:1011700089C32DF18AC32EF18BC32FF18CC330F1BB
:101180008DC331F18EC332F18FC333F10101296B6D
:1011900066EC16F0DDEC15F000C1AFFF01C1B0FF49
:1011A0001E0E0C6EAFCF0BF090EC06F01F0E0C6E07
:1011B000B0CF0BF090EC06F086EF0FF080B6E8EFC2
:1011C00008F00401300E826F8FEC08F0EDEF08F0AC
:1011D0000401310E826F8FEC08F099EC08F086EF75
:1011E0000FF083C32AF184C32BF185C32CF186C38E
:1011F0002DF187C32EF188C32FF189C330F18AC343
:1012000031F18BC332F18CC333F1010166EC16F07E
:10121000DDEC15F0160E0C6E00C10BF090EC06F034
:10122000170E0C6E01C10BF090EC06F0180E0C6E50
:1012300002C10BF090EC06F0190E0C6E03C10BF01E
:1012400090EC06F000C18AF101C18BF102C18CF172
:1012500003C18DF100C18EF101C18FF102C190F186
:1012600003C191F1D3EF09F083C32AF184C32BF1B9
:1012700085C32CF186C32DF187C32EF188C32FF1CE
:1012800089C330F18AC331F18BC332F18CC333F19E
:10129000010166EC16F0DDEC15F000C18AF101C128
:1012A0008BF102C18CF103C18DF100C18EF101C13E
:1012B0008FF102C190F103C191F1D3EF09F083C323
:1012C0002AF184C32BF185C32CF186C32DF187C38A
:1012D0002EF188C32FF189C330F18AC331F18CC359
:1012E00032F18DC333F1010166EC16F0DDEC15F03F
:1012F0000101000E046F000E056F010E066F000E57
:10130000076F2EEC15F01A0E0C6E00C10BF090EC6E
:1013100006F01B0E0C6E01C10BF090EC06F01C0EDB
:101320000C6E02C10BF090EC06F01D0E0C6E03C1AA
:101330000BF090EC06F000C192F101C193F102C1F3
:1013400094F103C195F1D3EF09F083C32AF184C36B
:101350002BF185C32CF186C32DF187C32EF188C3F1
:101360002FF189C330F18AC331F18CC332F18DC3BF
:1013700033F1010166EC16F0DDEC15F00101000E11
:10138000046F000E056F010E066F000E076F2EEC46
:1013900015F000C192F101C193F102C194F103C1B2
:1013A00095F1D3EF09F0160EA7EC06F0E8CF00F1A7
:1013B000170EA7EC06F0E8CF01F1180EA7EC06F027
:1013C000E8CF02F1190EA7EC06F0E8CF03F1BBEC71
:1013D00015F09EEC13F00401730E826F8FEC08F091
:1013E00004012C0E826F8FEC08F08AC100F18BC1D2
:1013F00001F18CC102F18DC103F1BBEC15F09EEC43
:1014000013F00401730E826F8FEC08F004012C0EB0
:10141000826F8FEC08F01A0EA7EC06F0E8CF00F10F
:101420001B0EA7EC06F0E8CF01F11C0EA7EC06F0AE
:10143000E8CF02F11D0EA7EC06F0E8CF03F1A1EC16
:101440000FF004012C0E826F8FEC08F092C100F1B6
:1014500093C101F194C102F195C103F1A1EC0FF028
:1014600099EC08F086EF0FF00401690E826F8FECA3
:1014700008F004012C0E826F8FEC08F00101040EBD
:10148000006F000E016F000E026F000E036FBBECC9
:1014900015F02CC182F40401300E82278FEC08F085
:1014A0002DC182F40401300E82278FEC08F02EC18A
:1014B00082F40401300E82278FEC08F02FC182F4F1
:1014C0000401300E82278FEC08F030C182F4040151
:1014D000300E82278FEC08F031C182F40401300E07
:1014E00082278FEC08F032C182F40401300E82278B
:1014F0008FEC08F033C182F40401300E82278FECA8
:1015000008F004012C0E826F8FEC08F00101050E2B
:10151000006F000E016F000E026F000E036FBBEC38
:1015200015F02CC182F40401300E82278FEC08F0F4
:101530002DC182F40401300E82278FEC08F02EC1F9
:1015400082F40401300E82278FEC08F02FC182F460
:101550000401300E82278FEC08F030C182F40401C0
:10156000300E82278FEC08F031C182F40401300E76
:1015700082278FEC08F032C182F40401300E8227FA
:101580008FEC08F033C182F40401300E82278FEC17
:1015900008F004012C0E826F8FEC08F00101210E7F
:1015A000006F000E016F000E026F000E036FBBECA8
:1015B00015F02CC182F40401300E82278FEC08F064
:1015C0002DC182F40401300E82278FEC08F02EC169
:1015D00082F40401300E82278FEC08F02FC182F4D0
:1015E0000401300E82278FEC08F030C182F4040130
:1015F000300E82278FEC08F031C182F40401300EE6
:1016000082278FEC08F032C182F40401300E822769
:101610008FEC08F033C182F40401300E82278FEC86
:1016200008F004012C0E826F8FEC08F0200EF86E8B
:10163000F76AF66A04010900F5CF82F48FEC08F02E
:101640000900F5CF82F48FEC08F00900F5CF82F4A1
:101650008FEC08F00900F5CF82F48FEC08F0090058
:10166000F5CF82F48FEC08F00900F5CF82F48FEC0F
:1016700008F00900F5CF82F48FEC08F00900F5CFEF
:1016800082F48FEC08F099EC08F086EF0FF08351AC
:10169000630AD8A486EF0FF08451610AD8A486EFBC
:1016A0000FF085516C0AD8A486EF0FF08651410ADD
:1016B0003FE08651440A1BE08651420AD8B4ABEFA2
:1016C0000BF08651350AD8B410EF11F08651360A66
:1016D000D8B465EF11F08651370AD8B4CEEF11F0C7
:1016E0008651380AD8B42CEF12F086EF0FF0079825
:1016F000079A04017A0E826F8FEC08F00401780ECD
:10170000826F8FEC08F00401640E826F8FEC08F09A
:101710000401550E826F8FEC08F094EF0BF004017A
:101720004C0E826F8FEC08F099EC08F086EF0FF00A
:101730000788079A04017A0E826F8FEC08F0040183
:10174000410E826F8FEC08F00401610E826F8FEC06
:1017500008F088EF0BF00798078A04017A0E826F71
:101760008FEC08F00401420E826F8FEC08F0040148
:10177000610E826F8FEC08F088EF0BF00101666755
:10178000C9EF0BF06767C9EF0BF06867C9EF0BF0A3
:101790006967E1EF0BF04F67D5EF0BF05067D5EFBE
:1017A0000BF05167D5EF0BF05267E1EF0BF0010141
:1017B000000E006F000E016F000E026F000E036F2F
:1017C00012000101620E046F010E056F000E066F1C
:1017D000000E076F66C100F167C101F168C102F137
:1017E00069C103F11DEC15F003BF65EF0CF00101B9
:1017F000000E046FA80E056F550E066F020E076FE0
:1018000066C100F167C101F168C102F169C103F16C
:1018100066C186F167C187F168C188F169C189F144
:101820001DEC15F003BF1EEF0CF00101000E866FDA
:10183000A80E876F550E886F020E896F0E0EA7ECEB
:1018400006F0E8CF18F10F0EA7EC06F0E8CF19F17B
:10185000100EA7EC06F0E8CF1AF1110EA7EC06F077
:10186000E8CF1BF166EC14F086C104F187C105F1E5
:1018700088C106F189C107F11DEC15F007822AEC39
:1018800014F066EC14F007922AEC14F086C100F113
:1018900087C101F188C102F189C103F107922AECE5
:1018A00014F0CC0E046FE00E056F870E066F050E68
:1018B000076F1DEC15F000C118F101C119F102C14B
:1018C0001AF103C11BF19DEF0CF00101800E006FB6
:1018D0001A0E016F060E026F000E036F4FC104F166
:1018E00050C105F151C106F152C107F11DEC15F0CF
:1018F00003AF7EEF0CF018EC16F012000E0EA7EC02
:1019000006F0E8CF18F10F0EA7EC06F0E8CF19F1BA
:10191000100EA7EC06F0E8CF1AF1110EA7EC06F0B6
:10192000E8CF1BF14FC100F150C101F151C102F1EB
:1019300052C103F107822AEC14F018C100F119C159
:1019400001F11AC102F11BC103F112000401730E6F
:10195000826F8FEC08F004012C0E826F8FEC08F080
:10196000078462C166F163C167F164C168F165C152
:1019700069F14BC14FF14CC150F14DC151F14EC114
:1019800052F157C159F158C15AF10794CCEC0CF0FF
:1019900099EC08F086EF0FF066C100F167C101F124
:1019A00068C102F169C103F10101BBEC15F09EECC5
:1019B00013F00401630E826F8FEC08F004012C0E0B
:1019C000826F8FEC08F04FC100F150C101F151C19D
:1019D00002F152C103F10101BBEC15F09EEC13F0D2
:1019E0000401660E826F8FEC08F004012C0E826FEA
:1019F0008FEC08F018EC16F059C100F15AC101F152
:101A00000101BBEC15F09EEC13F00401740E826F23
:101A10008FEC08F0120010820401530E826F8FECDD
:101A200008F004012C0E826F8FEC08F083C32AF1BA
:101A300084C32BF185C32CF186C32DF187C32EF10E
:101A400088C32FF189C330F18AC331F18BC332F1DE
:101A50008CC333F1010166EC16F0DDEC15F000C12A
:101A600066F101C167F102C168F103C169F18EC37A
:101A70002AF18FC32BF190C32CF191C32DF192C3A6
:101A80002EF193C32FF194C330F195C331F196C376
:101A900032F197C333F1010166EC16F0DDEC15F07D
:101AA00000C14FF101C150F102C151F103C152F126
:101AB00059EC16F099C32FF19AC330F19BC331F161
:101AC0009CC332F19DC333F1010166EC16F0DDECED
:101AD00015F000C159F101C15AF1CCEC0CF0040130
:101AE0002C0E826F8FEC08F07DEF0DF08251520AC0
:101AF00003E10F827DEF0DF00F928251750A03E131
:101B0000108484EF0DF010948251550A03E1108681
:101B10008BEF0DF01096078410B2E8EF0DF010A4D3
:101B2000D4EF0DF0B6C166F1B7C167F1B8C168F185
:101B3000B9C169F1BAC16AF1BBC16BF1BCC16CF149
:101B4000BDC16DF1BEC16EF1BFC16FF1C0C170F119
:101B5000C1C171F1C2C172F1C3C173F1C4C174F1E9
:101B6000C5C175F1C6C176F1C7C177F1C8C178F1B9
:101B7000C9C179F1CAC17AF1CBC17BF1CCC17CF189
:101B8000CDC17DF1CEC17EF1CFC17FF1D0C180F159
:101B9000D1C181F1D2C182F1D3C183F1D4C184F129
:101BA000D5C185F1DCEF0DF062C166F163C167F16B
:101BB00064C168F165C169F14BC14FF14CC150F18D
:101BC0004DC151F14EC152F157C159F158C15AF1AD
:101BD00007940FA00AEF0EF001019267F7EF0DF0E6
:101BE0009367F7EF0DF09467F7EF0DF09567FBEF54
:101BF0000DF00AEF0EF0BEEC0BF092C104F193C1B0
:101C000005F194C106F195C107F11DEC15F003BF74
:101C10004EEF0FF0BEEC0BF00101000E046F000E52
:101C2000056F010E066F000E076F4EEC15F010A445
:101C300021EF0EF00401750E826F8FEC08F026EF95
:101C40000EF00401720E826F8FEC08F004012C0E6E
:101C5000826F8FEC08F0BBEC15F0296735EF0EF0C2
:101C60000401200E826F38EF0EF004012D0E826FFA
:101C70008FEC08F030C182F40401300E82278FEC23
:101C800008F031C182F40401300E82278FEC08F095
:101C900004012E0E826F8FEC08F032C182F4040131
:101CA000300E82278FEC08F033C182F40401300E2D
:101CB00082278FEC08F004016D0E826F8FEC08F024
:101CC00004012C0E826F8FEC08F04FC100F150C15F
:101CD00001F151C102F152C103F10101BBEC15F058
:101CE0009EEC13F00401480E826F8FEC08F00401A3
:101CF0007A0E826F8FEC08F004012C0E826F8FEC4D
:101D000008F066C100F167C101F168C102F169C163
:101D100003F10101BBEC15F09EEC13F00401630E1E
:101D2000826F8FEC08F004012C0E826F8FEC08F0AC
:101D300066C100F167C101F168C102F169C103F137
:101D400001010A0E046F000E056F000E066F000EF3
:101D5000076F2EEC15F0000E046F120E056F000ECB
:101D6000066F000E076F4EEC15F0BBEC15F02AC1A4
:101D700082F40401300E82278FEC08F02BC182F42C
:101D80000401300E82278FEC08F02CC182F404018C
:101D9000300E82278FEC08F02DC182F40401300E42
:101DA00082278FEC08F02EC182F40401300E8227C6
:101DB0008FEC08F02FC182F40401300E82278FECE3
:101DC00008F030C182F40401300E82278FEC08F055
:101DD00004012E0E826F8FEC08F031C182F40401F1
:101DE000300E82278FEC08F032C182F40401300EED
:101DF00082278FEC08F033C182F40401300E822771
:101E00008FEC08F00401730E826F8FEC08F0040170
:101E10002C0E826F8FEC08F018EC16F059C100F10F
:101E20005AC101F1B0EC10F00FB21AEF0FF00FA091
:101E30004CEF0FF004012C0E826F8FEC08F0200E97
:101E4000F86EF76AF66A04010900F5CF82F48FECA8
:101E500008F00900F5CF82F48FEC08F00900F5CF07
:101E600082F48FEC08F00900F5CF82F48FEC08F0D3
:101E70000900F5CF82F48FEC08F00900F5CF82F469
:101E80008FEC08F00900F5CF82F48FEC08F0090020
:101E9000F5CF82F48FEC08F099EC08F00F9086EF04
:101EA0000FF00401630E826F8FEC08F004012C0E1A
:101EB000826F8FEC08F08CEC0FF004012C0E826F17
:101EC0008FEC08F0FFEC0FF004012C0E826F8FEC0A
:101ED00008F07BEC10F004012C0E826F8FEC08F000
:101EE0000101F80E006FCD0E016F660E026F030E3A
:101EF000036FA1EC0FF004012C0E826F8FEC08F041
:101F000091EC10F099EC08F086EF0FF00301C26B32
:101F10000790109295EF12F0D8900E0EA7EC06F0F5
:101F2000E8CF00F10F0EA7EC06F0E8CF01F1100E9C
:101F3000A7EC06F0E8CF02F1110EA7EC06F0E8CF0F
:101F400003F10101000E046F000E056F010E066F14
:101F5000000E076F4EEC15F0BBEC15F02AC182F4B1
:101F60000401300E82278FEC08F02BC182F40401AB
:101F7000300E82278FEC08F02CC182F40401300E61
:101F800082278FEC08F02DC182F40401300E8227E5
:101F90008FEC08F02EC182F40401300E82278FEC02
:101FA00008F02FC182F40401300E82278FEC08F074
:101FB00030C182F40401300E82278FEC08F031C169
:101FC00082F40401300E82278FEC08F004012E0EFB
:101FD000826F8FEC08F032C182F40401300E822748
:101FE0008FEC08F033C182F40401300E82278FECAD
:101FF00008F004016D0E826F8FEC08F01200120ED3
:10200000A7EC06F0E8CF00F1130EA7EC06F0E8CF3E
:1020100001F1140EA7EC06F0E8CF02F1150EA7ECC3
:1020200006F0E8CF03F101010A0E046F000E056F00
:10203000000E066F000E076F2EEC15F0000E046FF9
:10204000120E056F000E066F000E076F4EEC15F0B6
:10205000BBEC15F02AC182F40401300E82278FEC0C
:1020600008F02BC182F40401300E82278FEC08F0B7
:102070002CC182F40401300E82278FEC08F02DC1B0
:1020800082F40401300E82278FEC08F02EC182F416
:102090000401300E82278FEC08F02FC182F4040176
:1020A000300E82278FEC08F030C182F40401300E2C
:1020B00082278FEC08F004012E0E826F8FEC08F05F
:1020C00031C182F40401300E82278FEC08F032C156
:1020D00082F40401300E82278FEC08F033C182F4C1
:1020E0000401300E82278FEC08F00401730E826F1A
:1020F0008FEC08F012000A0EA7EC06F0E8CF00F112
:102100000B0EA7EC06F0E8CF01F10C0EA7EC06F0E1
:10211000E8CF02F10D0EA7EC06F0E8CF03F1B0EF27
:1021200010F0060EA7EC06F0E8CF00F1070EA7ECC2
:1021300006F0E8CF01F1080EA7EC06F0E8CF02F1B7
:10214000090EA7EC06F0E8CF03F1B0EF10F00101A3
:1021500018EC16F0078457C100F158C101F107943B
:102160000101E80E046F800E056F000E066F000E71
:10217000076F2EEC15F0000E046F040E056F000EB5
:10218000066F000E076F4EEC15F0880E046F130EED
:10219000056F000E066F000E076F1DEC15F00A0E9E
:1021A000046F000E056F000E066F000E076F4EECF9
:1021B00015F0BBEC15F001012967E4EF10F0040104
:1021C000200E826FE7EF10F004012D0E826F8FEC6E
:1021D00008F030C182F40401300E82278FEC08F041
:1021E00031C182F40401300E82278FEC08F032C135
:1021F00082F40401300E82278FEC08F004012E0EC9
:10220000826F8FEC08F033C182F40401300E822714
:102210008FEC08F00401430E826F8FEC08F012007F
:1022200087C32AF188C32BF189C32CF18AC32DF10E
:102230008BC32EF18CC32FF18DC330F18EC331F1DE
:1022400090C332F191C333F10101296B66EC16F0B2
:10225000DDEC15F00101000E046F000E056F010E9C
:10226000066F000E076F2EEC15F00E0E0C6E00C1FF
:102270000BF090EC06F00F0E0C6E01C10BF090EC21
:1022800006F0100E0C6E02C10BF090EC06F0110E71
:102290000C6E03C10BF090EC06F004017A0E826F15
:1022A0008FEC08F004012C0E826F8FEC08F0040113
:1022B000350E826F8FEC08F004012C0E826F8FECCC
:1022C00008F08CEC0FF094EF0BF087C32AF188C371
:1022D0002BF189C32CF18AC32DF18BC32EF18CC352
:1022E0002FF18DC330F18EC331F190C332F191C320
:1022F00033F10101296B66EC16F0DDEC15F0880E68
:10230000046F130E056F000E066F000E076F22ECB0
:1023100015F0000E046F040E056F000E066F000E20
:10232000076F2EEC15F00101E80E046F800E056FAB
:10233000000E066F000E076F4EEC15F00A0E0C6EC5
:1023400000C10BF090EC06F00B0E0C6E01C10BF00F
:1023500090EC06F00C0E0C6E02C10BF090EC06F047
:102360000D0E0C6E03C10BF090EC06F004017A0E1A
:10237000826F8FEC08F004012C0E826F8FEC08F056
:102380000401360E826F8FEC08F004012C0E826F70
:102390008FEC08F07BEC10F094EF0BF087C32AF180
:1023A00088C32BF189C32CF18AC32DF18BC32EF185
:1023B0008CC32FF18DC330F18FC331F190C332F153
:1023C00091C333F1010166EC16F0DDEC15F0000E5F
:1023D000046F120E056F000E066F000E076F2EECD5
:1023E00015F001010A0E046F000E056F000E066F56
:1023F000000E076F4EEC15F0120E0C6E00C10BF0C4
:1024000090EC06F0130E0C6E01C10BF090EC06F090
:10241000140E0C6E02C10BF090EC06F0150E0C6E53
:1024200003C10BF090EC06F004017A0E826F8FEC82
:1024300008F004012C0E826F8FEC08F00401370EB7
:10244000826F8FEC08F004012C0E826F8FEC08F085
:10245000FFEC0FF094EF0BF087C32AF188C32BF148
:1024600089C32CF18AC32DF18BC32EF18CC32FF1BC
:102470008DC330F18EC331F190C332F191C333F18A
:102480000101296B66EC16F0DDEC15F0880E046F87
:10249000130E056F000E066F000E076F22EC15F08D
:1024A000000E046F040E056F000E066F000E076F1E
:1024B0002EEC15F00101E80E046F800E056F000E82
:1024C000066F000E076F4EEC15F0060E0C6E00C185
:1024D0000BF090EC06F0070E0C6E01C10BF090ECC7
:1024E00006F0080E0C6E02C10BF090EC06F0090E1F
:1024F0000C6E03C10BF090EC06F004017A0E826FB3
:102500008FEC08F004012C0E826F8FEC08F00401B0
:10251000380E826F8FEC08F004012C0E826F8FEC66
:1025200008F091EC10F094EF0BF007A809EF13F00E
:102530000101800E006F1A0E016F060E026F000E71
:10254000036F4BC104F14CC105F14DC106F14EC101
:1025500007F11DEC15F003BF50EF13F098EC13F0EA
:102560004BC100F14CC101F14DC102F14EC103F16B
:1025700007822AEC14F018C104F119C105F11AC13F
:1025800006F11BC107F1F80E006FCD0E016F660E4C
:10259000026F030E036F1DEC15F00E0E0C6E00C1E2
:1025A0000BF090EC06F00F0E0C6E01C10BF090ECEE
:1025B00006F0100E0C6E02C10BF090EC06F0110E3E
:1025C0000C6E03C10BF090EC06F00784010118ECCF
:1025D00016F057C100F158C101F107940A0E0C6EB4
:1025E00000C10BF090EC06F00B0E0C6E01C10BF06D
:1025F00090EC06F00C0E0C6E02C10BF090EC06F0A5
:102600000D0E0C6E03C10BF090EC06F0079850EF26
:1026100013F007AA50EF13F00784010118EC16F02D
:1026200057C100F158C101F10794060E0C6E00C1AC
:102630000BF090EC06F0070E0C6E01C10BF090EC65
:1026400006F0080E0C6E02C10BF090EC06F0090EBD
:102650000C6E03C10BF090EC06F0078462C100F130
:1026600063C101F164C102F165C103F10794120E67
:102670000C6E00C10BF090EC06F0130E0C6E01C155
:102680000BF090EC06F0140E0C6E02C10BF090EC07
:1026900006F0150E0C6E03C10BF090EC06F0079AD5
:1026A0000401805181197F0B0BE09EA809D014EE24
:1026B00000F081517F0BE126E750812B0F01AD6EB9
:1026C000FBEF07F018C100F119C101F11AC102F1C5
:1026D0001BC103F1000E046F000E056F010E066FA3
:1026E000000E076F4EEC15F029A18DEF13F020516D
:1026F000D8B48DEF13F018C100F119C101F11AC15E
:1027000002F11BC103F1000E046F000E056F0A0EEB
:10271000066F000E076F4EEC15F012000101045118
:102720000013055101130651021307510313120040
:102730000101186B196B1A6B1B6B12002AC182F412
:102740000401300E82278FEC08F02BC182F40401C3
:10275000300E82278FEC08F02CC182F40401300E79
:1027600082278FEC08F02DC182F40401300E8227FD
:102770008FEC08F02EC182F40401300E82278FEC1A
:1027800008F02FC182F40401300E82278FEC08F08C
:1027900030C182F40401300E82278FEC08F031C181
:1027A00082F40401300E82278FEC08F032C182F4EB
:1027B0000401300E82278FEC08F033C182F404014B
:1027C000300E82278FEC08F012002FC182F4040132
:1027D000300E82278FEC08F030C182F40401300EF5
:1027E00082278FEC08F031C182F40401300E822779
:1027F0008FEC08F032C182F40401300E82278FEC96
:1028000008F033C182F40401300E82278FEC08F007
:102810001200060E116E060E126E060E136E112EAB
:102820000FEF14F0122E0FEF14F0132E0FEF14F021
:102830008B84020E116E020E126E020E136E112E9A
:102840001FEF14F0122E1FEF14F0132E1FEF14F0D1
:102850008B9412000101005305E1015303E102537F
:1028600001E1002BEDEC14F018EC16F03951006F7B
:102870003A51016F420E046F4B0E056F000E066F4A
:10288000000E076F2EEC15F000C104F101C105F137
:1028900002C106F103C107F118C100F119C101F12C
:1028A0001AC102F11BC103F107B25BEF14F022EC75
:1028B00015F05DEF14F01DEC15F000C118F101C129
:1028C00019F102C11AF103C11BF1120018EC16F044
:1028D00059C100F15AC101F1060EA7EC06F0E8CF8C
:1028E00004F1070EA7EC06F0E8CF05F1080EA7ECFF
:1028F00006F0E8CF06F1090EA7EC06F0E8CF07F1E5
:102900001DEC15F000C124F101C125F102C126F131
:1029100003C127F1290E046F000E056F000E066F2C
:10292000000E076F2EEC15F0EE0E046F430E056FD0
:10293000000E066F000E076F22EC15F024C104F1A3
:1029400025C105F126C106F127C107F12EEC15F0CE
:1029500000C11CF101C11DF102C11EF103C11FF133
:10296000120EA7EC06F0E8CF04F1130EA7EC06F068
:10297000E8CF05F1140EA7EC06F0E8CF06F1150E2E
:10298000A7EC06F0E8CF07F10D0E006F000E016F07
:10299000000E026F000E036F2EEC15F0180E046F80
:1029A000000E056F000E066F000E076F4EEC15F05F
:1029B0001CC104F11DC105F11EC106F11FC107F1C3
:1029C00022EC15F06A0E046F2A0E056F000E066FDA
:1029D000000E076F1DEC15F01200BF0EFA6E200EF0
:1029E0003A6F396BD8900037013702370337D8B0C8
:1029F000FEEF14F03A2FF3EF14F039073A070353C0
:102A0000D8B412000331070B80093F6F03390F0B55
:102A1000010F396F80EC5FF0406F390580EC5FF09B
:102A2000405D405F396B3F33D8B0392739333FA918
:102A300013EF15F040513927120001013DEC16F05B
:102A4000D8B01200010103510719346F00EC16F0E1
:102A5000D8900751031934AF800F12000101346B75
:102A600024EC16F0D8A03AEC16F0D8B012000FEC17
:102A700016F018EC16F01F0E366F50EC16F00B35F2
:102A8000D8B000EC16F0D8A00335D8B01200362F1D
:102A90003DEF15F034B127EC16F012000101346B54
:102AA00004510511061107110008D8A024EC16F0F6
:102AB000D8A03AEC16F0D8B01200086B096B0A6B7C
:102AC0000B6B50EC16F01F0E366F50EC16F00751E2
:102AD0000B5DD8A478EF15F006510A5DD8A478EF05
:102AE00015F00551095DD8A478EF15F00451085D83
:102AF000D8A08BEF15F00451085F0551D8A0053D13
:102B0000095F0651D8A0063D0A5F0751D8A0073DCE
:102B10000B5FD8900081362F65EF15F034B127ECAC
:102B200016F0346B24EC16F0D89054EC16F00751E4
:102B30000B5DD8A4A8EF15F006510A5DD8A4A8EF44
:102B400015F00551095DD8A4A8EF15F00451085DF2
:102B5000D8A0B7EF15F0003FB7EF15F0013FB7EF82
:102B600015F0023FB7EF15F0032BD8B4120034B1C3
:102B700027EC16F012000101346B24EC16F0D8B0EB
:102B8000120059EC16F0200E366F0037013702376D
:102B9000033711EE33F00A0E376FE7360A0EE75CA3
:102BA000D8B0E76EE552372FCDEF15F0362FC5EFD1
:102BB00015F034B12981D890120001010A0E346F4A
:102BC000200E366F11EE29F03451376F0A0ED8906F
:102BD000E652D8B0E726E732372FE8EF15F0033397
:102BE000023301330033362FE2EF15F0E750FF0FC9
:102BF000D8A00335D8B0120029B127EC16F0120086
:102C0000045100270551D8B0053D01270651D8B021
:102C1000063D02270751D8B0073D03271200005197
:102C2000086F0151096F02510A6F03510B6F1200B7
:102C30000101006B016B026B036B12000101046B5D
:102C4000056B066B076B12000335D8A01200035109
:102C5000800B001F011F021F031F003F37EF16F0FC
:102C6000013F37EF16F0023F37EF16F0032B342BFE
:102C7000032512000735D8A012000751800B041F4E
:102C8000051F061F071F043F4DEF16F0053F4DEFD0
:102C900016F0063F4DEF16F0072B342B07251200D8
:102CA0000037013702370337083709370A370B3740
:102CB00012000101296B2A6B2B6B2C6B2D6B2E6B79
:102CC0002F6B306B316B326B336B120001012A5169
:102CD0000F0B2A6F2B510F0B2B6F2C510F0B2C6FDF
:102CE0002D510F0B2D6F2E510F0B2E6F2F510F0BE0
:102CF0002F6F30510F0B306F31510F0B316F32513D
:0C2D00000F0B326F33510F0B336F1200BA
:10BF0000E844F926000C160C2B0C3F0C520C640C68
:10BF1000760C860C960CA50CB30CC10CCF0CDC0C6B
:06BF2000E80CF40C000C1B
:00000001FF
